:10000000830100308A003B28FC0003088301E600DE
:10001000831203130B1D202805140B110000000090
:1000200000000000000000000000000000000000D0
:10003000000000000000000000000000051036284D
:100040000C1F29281F089F000C133308573E8100FE
:1000500036288C1C36288C10AC0A2C08FA3A031D62
:100060003428AC01A017A0162014201766088300BE
:10007000FC0E7C0E090022308400663048202030BF
:1000800084002230482083012D2B04068001840A3D
:100090000406031D452800348207DE341234E6349A
:1000A00076343A347C34FC341634FE347E34803476
:0A00B00080342A346A340E344E34D2
:10046C0083160313061783120800830106178316DD
:10047C0006138312080083010613831606138312D6
:10048C000800362241223230812236223230812A33
:10049C008301B3080319542AB303552AA110C410BD
:1004AC00080083013308963A03195E2AB30A5F2ABF
:1004BC00A110C41408008301A118AC1E692AAC1F3A
:1004CC00692A06140800061008008301A013B70A55
:1004DC0037083C3A031D0800B701D80A8F22FA2AC4
:1004EC0083018615851E00348614851E003406157E
:1004FC00851E003401348301E2006208E3006400CD
:10050C00000000000000000000000000E20B852A43
:10051C00080083015C085806031DA22A5D085906D1
:10052C00031DA22A5E085A06031DA22A5F085B0659
:10053C00031DA22AA1140800A11008008301E001E8
:10054C0006138316061306176400000000008312BE
:10055C006108061FB32A0314B42A0310E10C0630F9
:10056C008122E00A08306002031CA62A61080800F8
:10057C008301E000E1010613601CCA2A83160613EE
:10058C00061706308122D02A8316061306308122E4
:10059C008316061703108312E00CE10A083061027F
:1005AC0003180800C12A8301A012A20A22082B06F4
:1005BC00031D0800A20147084F02031C4E2A4B08DA
:1005CC004702031C572A46084E02031C4E2A4A08AF
:1005DC004602031C572A45084D02031C4E2A4908A3
:1005EC004502031C57220800830158080A3A031DD0
:1005FC00032BD8012118032BD90A5908063A031DDD
:10060C00162BD9012118162BDA0A5A08043A031DA5
:10061C00162B5B08023A031D162BDA01DB010800CE
:10062C005A080A3A031D1E2BDA0121181E2BDB0A6D
:10063C005A08FC390319282B5B08023A031D282B96
:10064C00DB0108005B08033A0319DB010800652491
:10065C0076220038031D342B2111352B211521193D
:10066C00482BAB23201F3B2BFB25A01E3E2BD92256
:10067C00A01F412B0024A01F442B6B22211C372BC5
:10068C00FA22372B3808E0003908E1004830E20044
:10069C00E301E30AD4243A08E0003B08E1004C30C3
:1006AC00E200E301E30AD4242B08E000E10150301E
:1006BC00E200E301E30AD424AB23201F622BFB25C9
:1006CC00622B8301E200E401E501E301742BE830C5
:1006DC00E4070318E50A0330E507E30A6208033E62
:1006EC008400831300086302031C6D2BE301620872
:1006FC00023E840083130008630203188B2B6430C2
:10070C00E4070318E50AE30A7D2BE301620A84007F
:10071C008313000863020318992B0A30E4070318AB
:10072C00E50AE30A8C2BE3016208840083130008BA
:10073C0063020318A62BE40A0319E50AE30A9A2BB1
:10074C006508F1006408F000080061222010861191
:10075C00AD0A2D08043A031DB92BAD01211DB82B90
:10076C00D726B92B62258611211CC72B2D083606DE
:10077C000319AC1FC72B0616861686170516861589
:10078C00080000308A0032082D07443E8400831391
:10079C0000084C20E100AC1B61140611E001E11FC4
:1007AC00D92B0615DA2B061186140310E10D8610D1
:1007BC00E00A08306002031CD52B061186100616C1
:1007CC008616861705168615F32B06120800861258
:1007DC00080086130800051208002D080319EB2BDE
:1007EC00013A0319ED2B033A0319EF2B013A031DC0
:0407FC000800F12BD5
:100800008301D008031D0C2CD108031D0C2CD20829
:10081000031D0C2C85110800D408031D172CD508C6
:10082000031D172CD608031D172C85150800851DE0
:100830003C2CA70A27080A3A031D2A2CA701A80A5C
:1008400028080A3A031D2A2CA801A90A29080A3AED
:100850000319A90150082706031D0800510828069E
:10086000031D080052082906031D0800A701A8015E
:10087000A901851144100800A60A26083C3A031D68
:100880000800A601A30A23080A3A031D532CA3015A
:10089000A40A24080A3A031D532CA401A50A25081A
:1008A0000A3A0319A50154082306031D0800550838
:1008B0002406031D080056082506031D0800A30191
:1008C000A401A50185154414080005308312031303
:1008D0009F002630831685004030860083128501F4
:1008E0008601C53083168100811281118B16063076
:1008F00083129200F930831692008C1483121F0821
:100900009F000C1383160C170B178B174B30831299
:10091000B300B201AD01B601E830BA000330BB004C
:10092000B801B9012110A0142012A0112011043027
:10093000E000600883169B001C1483126008443E8C
:100940008400831383161A0880008312E00A1C3087
:100950006002031C992C0C30C4001D3083169B00D0
:100960001C141A088312B900B8011C3083169B00AE
:100970001C141A088312B8041F3083169B001C1421
:100980001A088312BB00BA011E3083169B001C1488
:100990001A088312BA04203083169B001C141A080C
:1009A0008312AB00A20108008301620A8400831352
:1009B00080016208023E8400831380016208033EC6
:1009C0008400831380011830E0070318E10AFC302B
:1009D000E1076208033E84008313800A6108803ABD
:1009E000F000803070020130031960020318E32C1C
:1009F000E11F052DE830E0070318E10A0330E107A5
:100A00006208033E8400831380039C30E007031CCC
:100A1000E1036208023E84008313800A6108803A81
:100A2000F000803070020130031960020318052DB8
:100A3000E11F232D6430E0070318E10A6208023E3B
:100A4000840083138003F630E007031CE103620A8D
:100A500084008313800A6108803AF00080307002BD
:100A60000130031960020318232DE11F3F2D0A30C6
:100A7000E0070318E10A620A840083138003E30895
:100A8000031908006208840083138001FF30E00727
:100A9000031CE103620884008313800A6108803A22
:100AA000F000803070020130031960020318462DF7
:100AB000E11F0800E00A0319E10A620884008313B9
:100AC000800308008301AA0A2A08043A0319AA012C
:100AD000AA08031D882D8615851AA01C822DA0103A
:100AE000A01521140310B20C0310B20CB20A320884
:100AF000073A031D7D2DB20121100310B20D031022
:100B0000B20D0800851EA01D0800A014A011080049
:100B10002A0BA42D8614851AA01C9E2DA010201629
:100B2000211C962DB60A0330B6050800B208031D35
:100B30009C2D1430B2000800B2010800851E201E52
:100B40000800A014201208002A08033A031D080018
:100B50000615851AA01CF52DA0102015A110211C2A
:100B6000080032083607443E84008313800A3208A6
:100B70003607443E8400831300080A3A031DC62D3D
:100B800032083607443E84008313800183169C1884
:100B9000C72D83123208360783169B008312320852
:100BA0003607443E84008313000883169A0003101E
:100BB0008B1B03148B131C1555309D00AA309D0010
:100BC0009C141C1103188B17831232080C3A031D56
:100BD000ED2DA701A801A90108003208103A031D54
:100BE0000800A301A401A5010800851E201D08001E
:100BF000A0142011080083012013B50A3508023A19
:100C0000031D0800B50121180800B4080319232E9C
:100C1000340B0B2E292E3408023A031D112EBE3040
:100C20002A2E3408033A031D182EA422B000D52E14
:100C30003408043A031D1F2EA422AE00D52E34081A
:100C4000053A031D252E4722D52E3408063A031DEA
:100C50002C2ECC30BE22D52E3408073A031D342E5C
:100C60004430BE223B22D52E3408083A031DBE2E46
:100C70002E08F300F2013008F000F1017208F004D0
:100C80007308F104700871080030F11BFF30F200A6
:100C9000F3007008C0007108C1007208C200730838
:100CA000C3003A08F4003B08F500F601F7014030B4
:100CB00084008313B727831203134108C00042083E
:100CC000C1004308C200C301F430C0070130031162
:100CD0000318013E031DC107003003110318013E34
:100CE000031DC207003003110318013E031DC30793
:100CF0003908F1003808F000F201F301C002710870
:100D0000031C710FC1027208031C720FC202730828
:100D1000031C730AC3023D08F1003C08F0004008C0
:100D2000F002031CF1034108F1027108803AF2005D
:100D3000843072020130031970020318B32E410887
:100D4000F1004008F0003C08F002031CF1033D08EC
:100D5000F1027108803AF200843072020130031906
:100D60007002031CB52E0A30B4004008BC004108D4
:100D7000BD004208BE004308BF00D52E3408093A22
:100D8000031DD52E211DCD2E4008E0004108E100B5
:100D90004430E200E301E30AD42E4008E0004108B9
:100DA000E1004430E200E301D424B40A08008301E6
:100DB000AA0A2A08043A0319AA01AA08031DFD2E4B
:100DC0008615851AA01CF72EA010A015211403105B
:100DD000B20C0310B20CB20A3208043A031DF22E10
:100DE000B20121100310B20D0310B20DB52F851EF4
:100DF000A01DB52FA014A011B52F2A0B112F8614FA
:100E0000851AA01C0B2FA0102016211CB52FB60A86
:100E10000330B605B52F851E201EB52FA014201255
:100E2000B52F2A08033A031DB52F0615851AA01CF5
:100E3000B02FA0102015A110211CB52F32083607A5
:100E4000443E84008313800A32083607443E8400FF
:100E5000831300080A3A031D332F32083607443E35
:100E60008400831380013208043A031D5A2F48304E
:100E700067237008B8007108B90083169C183E2FCC
:100E80001C309B008312380883169A0003108B1BBA
:100E900003148B131C1555309D00AA309D009C1423
:100EA0001C1103188B179C18532F1D309B008312A5
:100EB0003908802F3208083A031D8F2F4C306723E2
:100EC0007008BA007108BB0083169C18652F1E308D
:100ED0009B0083123A0883169A0003108B1B03149D
:100EE0008B131C1555309D00AA309D009C141C11BD
:100EF00003188B179C187A2F1F309B0083123B0816
:100F000083169A0003108B1B03148B131C1555308A
:100F10009D00AA309D009C141C1103188B1783128E
:100F200032080C3A031D0800503067237008AB00EC
:100F300083169C18992F20309B0083122B08831650
:100F40009A0003108B1B03148B131C1555309D0046
:100F5000AA309D009C141C11031CB52F8B17B52FB4
:100F6000851E201DB52FA014201183120800000833
:100F7000F000840A0008F100840A0008F200840AE4
:100F80000008F300C42F84017008F8007108F9000C
:100F90007208FA007308FB00F201F301F001F1019D
:100FA0000310FB0CFA0CF90CF80C031CE52F740869
:100FB000F00775080318750FF10776080318760F08
:100FC000F20777080318770FF307780879047A0493
:100FD0007B040319F12F0310F40DF50DF60DF70D39
:100FE000D02F84080319003473088000840372082A
:100FF000800084037108800084037008800000343E
:02400E00093F68
:10420000000000000000000005000500050003009C
:10421000050005000500030000000100000000008B
:10422000010000000000000000000000020001008A
:104230000500050005000500F4000100400006002F
:104240000A00000000000000000000000000000064
:00000001FF
